:020000040800F2
:10000000E0060020A10100089B300008952C0008A4
:1000100099300008B5040008BD3B0008000000004E
:100020000000000000000000000000001134000883
:100030008B060008000000009D300008B73400085F
:10004000BB010008BB010008BB01000849320008E1
:10005000BB010008BB010008BB010008BB01000890
:10006000BB010008BB010008BB010008BB01000880
:10007000BB010008BB0100082D0600083906000876
:10008000BB010008BB010008BB010008BB01000860
:10009000BB010008BB010008BB010008BB01000850
:1000A000BB010008BB010008BB010008BB01000840
:1000B000BB0100080000000000000000BB010008B8
:1000C000BB010008BB010008BB010008BB01000820
:1000D000BB010008813B0008BB010008BB01000810
:1000E000BB010008BB010008000000000000000088
:1000F0000000000000000000000000000000000000
:1001000000000000BB01000800000000BB01000867
:100110000000000000000000BB010008BB01000857
:10012000BB010008BB010008BB010008BB010008BF
:10013000BB010008000000000000000000000000FB
:10014000BB010008BB010008BB0100080000000063
:100150004506000851060008512E0008BB010008A2
:10016000BB010008BB010008BB0100080000000043
:10017000BB010008BB0100080000000000000000F7
:10018000BB010008BB010008BB010008DFF80CD070
:1001900000F07EF800480047493C0008E0060020D7
:1001A0000648804706480047FEE7FEE7FEE7FEE711
:1001B000FEE7FEE7FEE7FEE7FEE7FEE7353500086F
:1001C0008D0100082DE9F05F0546002092469B4610
:1001D00088460646814640241BE02846414647465D
:1001E000224600F044F853465A46C01A914110D3B3
:1001F00011461846224600F02BF82D1A67EB01082D
:100200004F4622460120002100F022F817EB00099A
:100210004E41201EA4F10104DFDC484631462A4647
:10022000434600F000B830BCBDE8C09FD2B201E048
:1002300000F8012B491EFBD270470022F6E710B5EB
:1002400013460A4604461946FFF7F0FF204610BD44
:10025000202A04DB203A00FA02F100207047914086
:10026000C2F1200320FA03F3194390407047202A7B
:1002700004DB203A21FA02F00021704721FA02F350
:10028000D040C2F120029140084319467047000057
:10029000064C074D06E0E06840F0010394E80700D3
:1002A00098471034AC42F6D3FFF774FF303E000895
:1002B000503E00082DE9F041044600270D46006835
:1002C00002F0A2FD0646206802F09AFD30435DD0A0
:1002D0002068C1682E4E890105D5617E012902D1B1
:1002E000217E01290BD0022D1DD0206802F08CFD4B
:1002F000B8B120688168C1F3400169B111E00125FE
:10030000244902E08F4232D27F1C0268D243520657
:10031000F8D440210160E8E78168314041F01001E4
:100320008160012D11D0206802F06AFD48B120687B
:100330008168C1F3400121B98168314041F0200159
:100340008160022D08D0032D04D0042501F0D6F9D8
:10035000064617E00C25F9E70825F7E701F0CEF986
:10036000801B05280ED92068806828420AD0606D5D
:1003700040F010006065A06D40F00100A065012014
:10038000BDE8F081206880682842E7D10020F7E7C7
:10039000C0FFFF7F000040A370B50446006881687D
:1003A0008268C1F3400112F0010F28D039BB816887
:1003B00001F00D01012914D18168124A1140891CF4
:1003C000816021680320086001F098F9054612E079
:1003D00001F094F9401B02280DD920688068C007FD
:1003E00009D0606D40F010006065A06D40F0010024
:1003F000A065012070BD20688068C007E8D100209A
:1004000070BD0000C0FFFF7FF8B5044600200090DB
:100410002068816811F0010F41D18168214A1142A1
:100420002ED18168D5432940491C81601E488068CF
:1004300000F0E07000020DD51C481D490068B0FBBB
:10044000F1F0401C00EB4000800000E0401E0090F6
:100450000028FBD101F052F906461BE0816811F03B
:10046000010F03D181682940491C816001F046F9E0
:10047000801B02280ED920680068C043C00709D03D
:10048000606D40F010006065A06D40F00100A06557
:100490000120F8BD20680168C943C907DED10020EA
:1004A000F8BD00003F000080000304502800002039
:1004B000400D0300FEE7000000EE100ADFED161A03
:1004C0009FED161AB8EE400A1649F0EE060A80EEC5
:1004D000212ADFED131A22EE011A81EE210A10EE15
:1004E000100A884201DC0020704710EE100A0E4905
:1004F000884201DB6420704770EE600A9FED0B1AA2
:1005000080EE810ADFED0A0A20EE200ABCEEC00A66
:1005100010EE100A80B2704700F07F4585EB714005
:1005200021B0F23E00003040666686409899B93F9F
:100530000000C84270B505464FF6FF7000224AF22F
:1005400001040EE0AB5C58400023C60702D084EAE9
:10055000500000E040085B1C9BB2082BF5D3521CF6
:1005600092B28A42EED370BD30B587B0142168468E
:10057000FFF763FE294CE06C40F00200E064E06CA1
:1005800000F002000590E06C40F00400E064E06CD4
:1005900000F004000590E06C40F08000E064E06C46
:1005A00000F080000590206E40F480402066206EB0
:1005B000694600F4804005900320019000200290DD
:1005C0004FF6F27000904FF0904000F0A1FF4FF610
:1005D000FF7569461248009500F09AFF6946114878
:1005E000009500F095FF69460F48009500F090FFD8
:1005F000E06C20F00200E064E06C20F00400E064B5
:10060000E06C20F08000E064E06C20F40050E064D6
:10061000206E20F48040206607B030BD00100240FC
:100620000004004800080048001C0048014800F091
:10063000C5BD000074020020014800F0BFBD0000ED
:100640002C020020014800F0B9BD0000E4010020A8
:10065000014800F0B3BD00009C01002030B590F8C7
:10066000444004F01C050124AC40056C6C60046837
:1006700063608368102B036803D099600068C260D0
:1006800030BD9A600068C16030BD7047F8B5FFF7B3
:100690006BFF4FF0E024206920F002002061206908
:1006A00020F001002061264DA86D40F08050A86523
:1006B000A86D00F080500090A86820F40040A86069
:1006C00000224FF400111F4801F0B6FE1D4E3068A5
:1006D000016841F010010160D5F8880040F44060E5
:1006E000C5F88800304601F077FE304601F08CFEF8
:1006F0003068016841F0020101603068816841F4AE
:1007000080018160012001F0D3F8206960F00200CF
:100710002061206960F0010020610A2000F044FEA1
:1007200002F0CCFE02F022FC074800F00BFA02F0C7
:10073000ABFB304601F00AFFBDE8F84002F070BCA8
:1007400000100240940000203000002072B6FEE746
:100750002DE9F84F00270446009790F85000DFF885
:10076000B0930D46B846012811D0012684F8506098
:10077000206802F049FB60B1606D40F020006065C8
:100780005FF0010784F85080384600F0D7B90220A6
:10079000FBE769680C20052912D8022907D0032934
:1007A00007D0042907D0052907D0062107E0686093
:1007B00006E0122103E0182101E04FF48071696026
:1007C000D5E90021236800EA91101844036B01F079
:1007D0001F014FF01F0C0CFA01FCC2F3846223EAE4
:1007E0000C038A4013430363206802F00DFB82462A
:1007F000206802F005FB5AEA00001DD1AA682968AA
:10080000206802F00DFB20686969C268C2F3C1026A
:10081000520091402A69042A0FD000EB82002B6815
:10082000026EDFF8F0C203F0F84302EA0C020B4359
:100830001A4342F00041016672E0002102F0DAFA48
:10084000400320684FF0000172D002F0D3FA90FA12
:10085000A0F0B0FA80F1286842036ED090FAA0F0C0
:10086000B0FA80F0814204D100221146206802F0E3
:10087000E6FA0121206802F0BDFA400320684FF03B
:1008800001015DD002F0B6FA90FAA0F0B0FA80F162
:100890002868420359D090FAA0F0B0FA80F0814263
:1008A00004D100220121206802F0C9FA0221206847
:1008B00002F0A0FA400320684FF0020148D002F095
:1008C00099FA90FAA0F0B0FA80F12868420344D077
:1008D00090FAA0F0B0FA80F0814204D10022022107
:1008E000206802F0ACFA0321206802F083FA40038A
:1008F00020684FF0030133D002F07CFA90FAA0F0A8
:10090000B0FA80F1286842032FD090FAA0F0B0FA34
:1009100080F0814204D100220321206802F08FFA86
:100920002068816811F0010F22D0ABE000E004E004
:1009300002F060FAC0F384618DE7C0F3846091E750
:1009400002F058FAC0F38461A2E7C0F38460A6E71E
:1009500002F050FAC0F38461B7E7C0F38460BBE7EC
:1009600002F048FAC0F38461CCE7C0F38460D0E7BA
:100970002A7B296850F8B03FC1F3120C23EA0C031C
:1009800002F0180C644A22FA0CF20A401343036086
:10099000E968494576D1286841031BD090FAA0F157
:1009A000B1FA81F1491C01F01F0109294FEA4031D8
:1009B00031D8002911D090FAA0F1B1FA81F100BF2D
:1009C00001F1010101F01F0106FA01F608D1C0F39F
:1009D000846109E0C0F38461E4E7C0F38461EFE778
:1009E00090FAA0F1B1FA81F101F1010101F01F01CA
:1009F00046EA816102D1C0F3846003E090FAA0F07E
:100A0000B0FA80F000F1010000F01F0000EB4000A0
:100A100041EA005132E000290ED090FAA0F1B1FA7B
:100A200081F100BF01F1010101F01F0106FA01F699
:100A300005D1C0F3846106E0C0F38461F2E790FA67
:100A4000A0F1B1FA81F101F1010101F01F0146EAC3
:100A5000816102D1C0F3846003E090FAA0F0B0FAA3
:100A600080F000F1010000F01F002C4A00EB400074
:100A700002EB005041EA000141F00071AA682068D1
:100A800002F0CEF926482A6802423FF47BAE2548A0
:100A90008168254D254B01F0E071AA421BD10D0262
:100AA00019D422689A427FF46DAE826841F4000145
:100AB00022F0E0720A4382601D481E490068B0FBC4
:100AC000F1F0401C00EB4000800000E0401E009070
:100AD0000028FBD156E6184DAA4207D1CD0105D416
:100AE00022689A42F6D141F080710AE06FF0004529
:100AF000EA42EFD14A02EDD422689A42EAD141F4A7
:100B00008001826822F0E0720A4382603AE60000C7
:100B100000007F4000F0FF03FFFF0700000020FE01
:100B20000000088000030450000052C70000045079
:100B300028000020400D0300000084CB18BCBDE855
:100B4000E08F000070B504000FD0606D40F002002F
:100B5000606503212046FFF7ADFB05002068C168F2
:100B600041F40011C16002D008E0012070BD2046B0
:100B7000FFF712FC050001D1012060652068416883
:100B80006FF30A014160216840F2FF70086020683D
:100B9000816821F0A04181602068816841F00051A6
:100BA00081602068C1683D4A1140C1602068C16809
:100BB00041F00041C160206801696FF30A010161E1
:100BC0002068416901F0404141612068816901F07C
:100BD000784181612068016A01F0F021016220689A
:100BE000416A01F0FF2141622068816A01F0FF2122
:100BF00081622068016B2A4A114001632068426BC0
:100C0000274910390A4042632068826B0A40826398
:100C10002068C16B40F2DF729143C16321680A6EA4
:100C2000204802400A6621684A6E02404A662168EE
:100C30008A6E02408A662168CA6E0240CA662068CF
:100C400050F8A01F6FF312010160206850F8A41F34
:100C50006FF312010160206850F8B01F6FF31201AA
:100C60000160206850F8B41F21F07F1101600E4828
:100C7000816811F0010F08D1D0F808130B4A114018
:100C8000C0F80813204600F0EFF80020A065E065EA
:100C90002066606584F85000284670BD048000809E
:100CA000300882E000F0FF0300000450FFFF00FE68
:100CB0000068006C70470000F8B54FF000050400B4
:100CC0002E46009502D0606D10B107E00120F8BDFE
:100CD000204600F0DDF8A66584F850602068816841
:100CE000C1F3407119B18168574A11408160206891
:100CF0008168C1F3007189B98168544A114041F09B
:100D000080518160524853490068B0FBF1F04000C7
:100D1000801C00E0401E00900028FBD12068816804
:100D2000C1F3007141B9616D41F010016165A16DC0
:100D300041F00101A165012502F066F8616D01F045
:100D400010010143606D05D040F010006065012581
:100D50002846F8BD20F4807040F0020060652068ED
:100D6000806810F0010F0BD13B48806810F0010F34
:100D700006D13A486168826822F47C120A43826094
:100D8000E168606B627E0843A16841EA4231084332
:100D900094F8201040EA0140012904D1A18C304A86
:100DA00002EB41410843A16A29B101F47071E26A82
:100DB000014342EA01002268D1682A4B19400143ED
:100DC000D160206802F020F80646206802F018F88A
:100DD000304315D1207E94F83010800340EA410260
:100DE0002068C16844F2020399431143C16094F83A
:100DF000380001280CD02068016921F0010101614F
:100E0000206901282068016B21F00F0111D013E047
:100E1000D4E90F010843D4E91112114308432168B2
:100E20000A6940F2FC739A43104340F001000861E4
:100E3000E6E7E269521E11430163606D20F0020093
:100E400040F00100606583E7C0FFFF5FC0FFFF7FE8
:100E500028000020400D030000000450000304504F
:100E60000000FEFF07C0F0FF00680749884209D173
:100E70000648C16C21F40051C16402214FF090403A
:100E800000F0A4BA704700000000045000100240B7
:100E900010B59EB00446142117A8FFF7CEF95C21C7
:100EA0006846FFF7CAF917492068884227D14FF4EE
:100EB000804000904FF040501490684600F02CFDA8
:100EC00008B1FFF743FC1048C16C41F40051C16404
:100ED000C16C01F400511C91C16C41F00101C1646D
:100EE000C06C17A900F001001C90022017900B2085
:100EF0001890002019904FF0904000F009FB1EB0B0
:100F000010BD000000000450001002402DE9F04127
:100F1000044640690E4608280AD02068C068C00709
:100F200008D0606D40F0200060650120BDE8F081D0
:100F3000082500E0042500F0E1FB074614E0701CE2
:100F400012D000F0DBFBC01BB04200D866B92068AD
:100F50000068284208D1606D40F004006065002000
:100F600084F850000320E1E7206800682842E6D0BA
:100F7000606D40F400706065206801F049FF80B149
:100F8000607E70B92068006800070AD5606D20F4A3
:100F900080706065606DC00403D4606D40F0010036
:100FA00060652068C168082D05D0490401D40C2172
:100FB00001600020BAE70821FAE7000010B50446F6
:100FC000006801F021FF10B10221084610BD94F81D
:100FD000500001280CD0012084F850002046FFF773
:100FE00013FA01004FF0000004D084F85000ECE741
:100FF000022010BD626D40F601639A4342F4807294
:101000006265626DD20404D5A26D22F00602A2656B
:1010100000E0A06523681C221A6084F85000206854
:10102000C268920105D5626D22F4005242F48052EA
:1010300062658268024B1A40121D8260C5E700009B
:10104000C0FFFF7F10B5044690F85000012808D07B
:10105000012084F8500003212046FFF72BF910B13E
:101060000BE0022010BD2046FFF796F928B9616D0C
:1010700021F4885141F001016165002184F850108C
:1010800010BD10B590F825100022022905D00421CA
:10109000C16380F82420012010BD01680B6823F093
:1010A0000E030B6001680B6823F001030B6090F8DE
:1010B0004410046C01F01C03012101FA03F3636086
:1010C00080F8251080F82420104610BD10B590F847
:1010D00025100024022903D00421C16301241AE051
:1010E00001680A6822F00E020A6001680A6822F0AC
:1010F00001020A6090F84410036C01F01C02012107
:1011000001FA02F25A6080F82510002180F82410BC
:10111000816B01B18847204610BD000030B590B109
:1011200001680A6822F001020A60204C0368142159
:101130001F4AA34209D21F4C1C44B4FBF1F18900A1
:10114000C0E910210BE0012030BD184C64421C4462
:10115000B4FBF1F1890041641449083901640021AC
:10116000196090F8443003F01C040123A340046C80
:101170006360046C0F23944202D152F8A84F02E03E
:101180000A4AA032146890F8445005F01C05AB40A0
:101190009C431460C162016341638163C16380F851
:1011A000251080F82410002030BD00000804024003
:1011B00000000240F8FFFDBFC06B7047F0B4016C47
:1011C0000C6801680D6890F8442002F01C060422A7
:1011D00002FA06F3234211D06B070FD50B689B066A
:1011E00003D40B6823F004030B6090F8441001F063
:1011F0001C018A40016C4A60016B1DE0022303FA66
:1012000006F727424FF0000C4FF0010218D0AF074D
:1012100016D50C68A40605D40C6824F00A040C60EA
:1012200080F8252090F8441001F01C018B40016CDF
:101230004B6080F824C0C16A00291AD0F0BC08476E
:101240000823B340234214D02B0712D50B6823F098
:101250000E030B6090F84410036C01F01C0102FABD
:1012600001F15960C26380F8252080F824C0416BE9
:10127000E2E7F0BC7047000070B568B12B4C036822
:1012800014212B4AA34209D22A4C1C44B4FBF1F18D
:101290008900C0E910210BE0012070BD234C64429D
:1012A0001C44B4FBF1F18900416420490839016410
:1012B000022180F825101C6847F6F0718C43D0E9B4
:1012C00002152943D0E9045635432943856929434A
:1012D000C5692943056A2943214319608168B1F52D
:1012E000804F19D0036C0F21934202D152F8A83FCE
:1012F00002E00E4AA032136890F8444004F01C0447
:10130000A1408B43136090F84430416803F01C0304
:1013100099401368194311600021C163012280F8CC
:10132000252080F82410084670BD00000804024003
:1013300000000240F8FFFDBF70B5044690F824009D
:10134000002501280CD0012084F8240094F82560A1
:101350000020012E06D084F824000225284670BD06
:10136000022070BD022684F82560E06320680668CC
:1013700026F0010606602046FFF770F9206B002872
:101380002068016802D041F00E0106E021F004015E
:1013900001602068016841F00A010160206801686D
:1013A00041F001010160D9E770B5044600F0A6F9EB
:1013B0000546601C02D004480078044400F09EF901
:1013C000401BA042FAD370BD1C0000202DE9F84F4D
:1013D00000230126DFF818C10F2782E006FA03F484
:1013E00014EA01027CD023F003056544AA46D5F82F
:1013F00008909D074FEA157E07FA0EF505EA090BDE
:101400000095B0F1904F05D03A4DA84205D14FF06C
:10141000010816E04FF0000813E0374DA84202D152
:101420004FF002080DE0354DA84202D14FF00308FD
:1014300007E0334DA84202D14FF0040801E04FF01D
:10144000070808FA0EF8D84526D1DFF8B880D8F892
:10145000009029EA0209C8F8009008F10408D8F8B9
:10146000009029EA0209C8F80090DFF8988008F196
:101470000C08D8F8009029EA0209C8F80090A8F1F1
:101480000408D8F800509543C8F80050009DDAF8D9
:101490000820AA43CAF80820D0F800804FEA430980
:1014A000032202FA09F248EA0208C0F80080DD08C7
:1014B00000EB8505AA46D5F820804FEA43794FEA2C
:1014C000D96907FA09F528EA0508CAF8208085686D
:1014D000954385604568A5434560C4689443C460EE
:1014E0005B1C31FA03F27FF479AF00F00DB8000015
:1014F000000001400004004800080048000C0048BB
:10150000001000480004014018BCBDE8E08F000056
:101510002DE9F04FDFF8AC9100230325A9F1040B6E
:1015200085B04FF0010C0F2709F1040AABF1040E4E
:10153000BFE000BF0CFA03F6324075D00C7904F01E
:101540000304012C01D0022C1BD1846800945C00A0
:1015500005FA04F80494009C24EA08040094D1F8E5
:101560000C80049C08FA04F8009C48EA0408C0F8BF
:1015700008804468B4430E79C6F300169E402643A3
:1015800046600C79E443A4070AD0C4684FEA4308D4
:1015900005FA08F6B4438E6806FA08F62643C660D4
:1015A0000C7904F00304022C10D1DC0800EB840455
:1015B0000294246A5E074FEAD66807FA08F6B44335
:1015C0000E6906FA08F62643029C266204684FEA72
:1015D000430805FA08F6B4430E7906F0030606FA46
:1015E00008F6264306604C6814F4403F60D0364C41
:1015F000266E46F001062666246E23F0030604F0EC
:1016000001040094314C34440294A4689E074FEACC
:10161000167807FA08F6B443B0F1904F05D02C4E77
:10162000B04204D1012612E042E000260FE0294E2C
:10163000B04201D102260AE0274EB04201D1032672
:1016400005E0264EB04201D1042600E0072606FA46
:1016500008F62643029CA660D9F800604C46D1F8F3
:10166000048096435FEAC82800D516432660DAF85E
:1016700000405646D1F8048094435FEA882800D59C
:1016800014433460DBF800405E46D1F80480944394
:101690005FEA883800D514433460DEF800407646AF
:1016A000D1F8048094435FEAC83800D5144334600D
:1016B0005B1C0A6832FA03F47FF43CAF05B000F01B
:1016C0000FB8000008040140001002400000014073
:1016D0000004004800080048000C004800100048C2
:1016E00030BCBDE8C08F0069084000D001207047C1
:1016F0000AB18161704781627047000001488068CB
:10170000704700001C0000200248816802781144E4
:10171000816070471C00002010B50024032000F0F9
:1017200081F80F2000F008F808B1012401E000F072
:1017300025F8204610BD000070B50E4E0546002469
:10174000307898B14FF47A71B1FBF0F00A4909682A
:10175000B1FBF0F000F02CFE40B9102D06D20022B3
:101760002946501E00F03EF8756000E00124204636
:1017700070BD00001C00002028000020094808B5AA
:10178000016E41F001010166016E01F0010100915D
:10179000816D41F080518165806D00F08050009036
:1017A00008BD00000010024000280DDB00F01F0201
:1017B000012191404009800000F1E020C0F8801133
:1017C000BFF34F8FBFF36F8F7047002809DB00F026
:1017D0001F02012191404009800000F1E020C0F883
:1017E00000117047F0B40E4B1B680C46C3F3022384
:1017F000C3F10705042D00D90425191D072901D2BD
:10180000002300E0DB1E012606FA05F1491E2140F7
:1018100099409E40761E16403143F0BC02F0D8B984
:101820000CED00E0064900F0070208684FF6FF03E0
:10183000184040EA0220034A104308607047000045
:101840000CED00E00000FA051649B0F5007F0868CD
:10185000C0F3412009D0022805D0086820F4C060F8
:1018600040F480600860002070470128FBD00868C1
:1018700020F4C06040F4007008600B483222006819
:1018800050430A4AB0FBF2F0401C00E0401E4A6997
:10189000520501D50028F9D148694005E3D5032058
:1018A00070470000007000402800002040420F00F8
:1018B0000B490A6822F00702921C0A6009490A686B
:1018C00042F004020A60012807D040BF20BF20BFB9
:1018D000086820F004000860704730BFF8E7000097
:1018E0000070004010ED00E00248006800F4C060A5
:1018F00070470000007000400248016841F48071A8
:1019000001607047007000400248016841F0040126
:1019100001607047001002402DE9F84F044600278F
:101920000088A84D3E46000515D5606C60B1B0F545
:10193000000F04D0B0F5400F2BD001270AE0E86873
:1019400040F48030E86024E00021201D01F0A8FB75
:1019500007001ED03E46206880033AD5A86D4FF0A0
:101960000008C00009D4A86D40F08050A865A86D9B
:101970004FF0010800F080500090DFF84CA2DAF838
:10198000001041F48071CAF80010FFF7B7FE8146DD
:1019900010E0D5F88800616C20F440000843C5F8D9
:1019A0008800D8E7FFF7AAFEA0EB0900022801D9BA
:1019B000032705E0DAF80000C005F3D5002F7DD03D
:1019C0004FEA0706B8F1000F03D0A86D20F0805051
:1019D000A8652078C00707D0D5F88800216A20F0D4
:1019E00003000843C5F888002078800707D5D5F89C
:1019F0008800616A20F00C000843C5F88800207850
:101A0000400707D5D5F88800A16A20F030000843C8
:101A1000C5F888002078800607D5D5F88800E16AE7
:101A200020F440600843C5F888002088800507D569
:101A3000D5F88800E16B20F440200843C5F8880001
:101A40002088400507D5D5F88800216C20F4401087
:101A50000843C5F888002078400607D5D5F88800E7
:101A6000216B20F440500843C5F888002078000618
:101A700007D5D5F88800616B20F440400843C5F8CD
:101A800088002088C00507D5D5F88800A16B20F410
:101A900040300843C5F8880020684FF00067000315
:101AA0004FF0806850D5D5F88800A16C20F04060D8
:101AB0000843C5F88800A06CB84200E005E03BD1BF
:101AC000E86840F48010E8603EE0D5F8900010F43B
:101AD000407014D0A16D814211D0D5F89000D5F896
:101AE000901020F4407041F48031C5F89010D5F882
:101AF000901021F48031C5F89010C5F89000C0070F
:101B000011D0FFF7FBFD074641F2883907E000BF1F
:101B1000FFF7F4FDC11B494501D9032652E7D5F86B
:101B200090008007F4D5D5F89000A16D20F44070A6
:101B30000843C5F8900045E7404505D10121201D27
:101B400001F0AEFA00B106462068400317D5D5F87B
:101B50008800E16C20F040600843C5F88800E06C24
:101B6000B84204D1E86840F48010E86007E04045DE
:101B700005D10121201D01F093FA00B1064620880D
:101B8000400411D5D5F88800216D20F0405008435D
:101B9000C5F88800206DB0F1805F05D10221201DBD
:101BA00001F07EFA00B106462088000406D555F8FB
:101BB000880F616D20F0804008432860304600F0B7
:101BC00005B80000001002400070004018BCBDE8DD
:101BD000E08F00002DE9F0470F4605006BD0494E1D
:101BE000306800F00700B84209D2306820F00700E2
:101BF00038433060306800F00700B8425BD1287885
:101C0000414C80070AD5A868A16801F0F00188421C
:101C100004D9A16821F0F0010143A1602878C00730
:101C20002CD06868032811D0022812D0216898B1FE
:101C3000490500293FDAA16821F003010143A160B1
:101C4000FFF75CFD804641F2883910E02168890188
:101C5000EFE721688903ECE78907EAE7FFF74EFD24
:101C6000A0EB0801494502D90320BDE8F087A06830
:101C7000696800F00C00B0EB810FEFD12878800785
:101C80000AD5A868A16801F0F001884204D2A168D1
:101C900021F0F0010143A160306800F00700B84274
:101CA0000BD9306820F0070038433060306800F00E
:101CB0000700B84201D00120D7E72878400705D5B2
:101CC000A068E96820F4E0600843A0602878000775
:101CD00006D5A068296920F4605040EAC100A060E0
:101CE00000F03EF8A168094AC1F30311515C01F00C
:101CF0001F01C8400649086006480068BDE8F04773
:101D0000FFF71ABD0020024000100240E83D000825
:101D10002800002020000020054806490068896846
:101D2000054AC1F30221515C01F01F01C840704710
:101D30002800002000100240283E000805480649FF
:101D400000688968054AC1F3C221515C01F01F0196
:101D5000C84070472800002000100240283E0008BC
:101D600070B52549002318468A68CC6812F00C0229
:101D700004F00306214C4FEA640509D00C2A05D073
:101D8000042A32D0082A00D1284670BD012E10D175
:101D90000B681B0704D4D1F89430C3F3032302E08B
:101DA0000B68C3F30313164E56F82330DAB10C2A2E
:101DB000EBD1C86800F00300022818D0032818D01F
:101DC0001846CA68CB68C2F30212C3F30623434322
:101DD000521CB3FBF2F2C868C0F34160401C4000E3
:101DE000B2FBF0F070BD184670BD204670BD2046B5
:101DF000E7E72846E5E70000001002400024F40071
:101E0000F83D00082DE9F84304006FD0FA4DA868AA
:101E100000F00C06E86800F003072078C00664D5DF
:101E200076B10C2E01D1012F0AD0A06900282868B4
:101E30007AD040F001002860FFF760FC80465DE04A
:101E40002868800702D5A0690028DED0216A2868AA
:101E5000000703D5286800F0F00004E0D5F89400EE
:101E6000F02202EA1010814216D9084601F0AEF9BC
:101E700000283BD1286840F0080028602868216AC3
:101E800020F0F000084328606868E16920F47F4092
:101E900040EA0120686016E0286840F008002860E9
:101EA0002868216A20F0F000084328606868E1692A
:101EB00020F47F4040EA0120686026B9206A01F0E2
:101EC00085F90028D5D1FFF74BFFA968CB4AC1F3AC
:101ED0000311515C01F01F01C840C9490860C9489D
:101EE0000068FFF729FC00287ED12EE0CAE000BF81
:101EF000FFF704FCA0EB0800022876D828688007CA
:101F0000F6D5286840F0080028602868216A20F08B
:101F1000F000084328606868E16920F47F4040EAE7
:101F20000120686011E0FFE720F001002860FFF762
:101F3000E5FB804606E000BFFFF7E0FBA0EB0800F2
:101F40000228DAD828688007F6D42078C00740D065
:101F5000082E18D00C2E01D1032F14D06068B0F5D4
:101F6000803F17D0B0F5A02F286817D020F480301C
:101F70002860286820F4802028606068E0B1FFF7BE
:101F8000BDFB804614E02868800322D560680028E5
:101F900078D01EE0286840F48030EDE740F48020DF
:101FA0002860F7E7FFF7AAFBA0EB08006428A4D895
:101FB00028688003F6D50CE0FFF7A0FB804605E01B
:101FC000FFF79CFBA0EB0800642896D828688003E4
:101FD000F6D4207880073BD5042E11D00C2E01D1E9
:101FE000022F0DD0E06801E0AAE1FFE00028286898
:101FF0001ED040F480702860FFF780FB07460CE09D
:10200000286840050CD5E0680028C1D008E000BF72
:10201000FFF774FBC01B022893D828684005F7D54A
:102020006868217C20F0F85040EA016068600FE0A9
:1020300020F480702860FFF761FB074605E000BFD1
:10204000FFF75CFBC01B0228B1D828684005F7D415
:102050002078000729D560690028D5F8940012D0AF
:1020600040F00100C5F89400FFF748FB074604E084
:10207000FFF744FBC01B022899D8D5F894008007CD
:10208000F6D512E02BE120F00100C5F89400FFF72F
:1020900035FB074605E000BFFFF730FBC01B0228F9
:1020A00085D8D5F894008007F6D42078400766D507
:1020B000A86D0027C00008D4A86D40F08050A86526
:1020C000A86D012700F0805000904F480168C905B5
:1020D00012D40168814641F480710160FFF70EFB64
:1020E000804605E0FFF70AFBA0EB080002287DD838
:1020F000D9F80000C005F5D5A068012816D005283C
:10210000D5F8900017D020F00100C5F89000D5F860
:10211000900020F0040000BFC5F89000A06841F2D4
:102120008839C0B1FFF7EAFA80460FE0D5F8900091
:1021300040F00100F0E740F00400C5F89000F5E73A
:10214000FFF7DCFAA0EB080149454FD8D5F890001D
:102150008007F5D50EE0FFF7D1FA804606E000BF14
:10216000FFF7CCFAA0EB080149453FD8D5F890001D
:102170008007F5D41FB1A86D20F08050A8652078A5
:10218000800628D5606A0028D5F8980012D040F063
:102190000100C5F89800FFF7B1FA074605E000BF57
:1021A000FFF7ACFAC01B022820D8D5F898008007AA
:1021B000F6D510E020F00100C5F89800FFF79EFA70
:1021C000074604E0FFF79AFAC01B02280ED8D5F89C
:1021D00098008007F6D4A06AF0B3022816D00C2E1F
:1021E0007DD0286820F08070286000E0A7E0FFF72D
:1021F00085FA0446A6E0000000100240E83D000811
:10220000280000202000002000700040E868E26AFA
:1022100000F00301914228D1216B00F07002090106
:102220001039914221D1626B00F4FE41B1EB022FD3
:102230001BD194F8382000F07841B1EBC26F14D173
:10224000A18F00F4C00249084905A1F5001191428F
:102250000BD194F8401000E06AE04908490600F00C
:10226000C060A1F1007181424BD00C2E73D0286860
:10227000400170D4286820F080702860FFF73EFA93
:10228000064604E0FFF73AFA801B022857D8286870
:102290008001F7D4F4E90B016FF00F0202EB01119A
:1022A0000843218A5204490802EB4151A26841EADD
:1022B00002210843217D4FF07E42490802EB416133
:1022C0000843217B40EAC160E968244A1140084381
:1022D000E860286840F080702860E86800E03AE034
:1022E00040F08070E860FFF709FA044605E000BF9F
:1022F000FFF704FA001B022821D828688001F7D5CF
:1023000027E02868800124D4286840F08070286085
:10231000E86840F08070E860FFF7F0F9044604E0F8
:10232000FFF7ECF9001B022809D828688001F7D5CF
:102330000FE000BFFFF7E2F9001B022802D90320DB
:10234000BDE8F88328688001F4D4E86804490840AF
:10235000E8600020F4E70120F2E700008C809D0196
:10236000FCFFEEFE00680349884202D102490120C9
:1023700008707047002800401400002010B50B4979
:1023800004464FF4801008602068C168490508D5EC
:10239000C16801F0800161F49061C1602046FFF7DF
:1023A000E1FF012084F8210010BD00001404014069
:1023B00010B5401EB0F1807F01D3012010BD4FF059
:1023C000E02460610F21601701F002FC0020A06191
:1023D00007202061002010BD90F87410012911D051
:1023E000012180F874100168083151E8002F42F48F
:1023F000000241E80023002BF5D1002180F8741081
:10240000084670470220704790F87410012910D0D8
:10241000012180F87410026852E8001F41F00201A7
:1024200042E80013002BF6D1002180F87410084612
:10243000704702207047704738B5044690F8740022
:102440000025012811D0012084F874002420A06701
:102450002068036823F0010303602068836823F485
:1024600040130B43836011B10EE0022038BD206899
:10247000416893B221F01001194341602068120CA9
:10248000416862F31F6141602068016841F0010109
:102490000160FFF733F903466FF07E4000900022A1
:1024A0004FF48001204601F007FB08B1032501E04D
:1024B0002020A067002084F87400284638BD7047AB
:1024C00070B50446806FE66F216889684FF010058B
:1024D000090618D5212816D12068083050E8001FB9
:1024E00021F0800140E80012002AF5D1E06E38B1F9
:1024F000FEF7C7FD20B1E06EFEF75EFE202821D07A
:10250000204601F07AF920688068400618D5222E0E
:1025100016D12068083050E8001F21F0400140E843
:102520000012002AF5D1206F38B1FEF7AAFD20B1C4
:10253000206FFEF741FE202804D0204601F038F934
:10254000002070BDC4F88050032070BD70B5040039
:1025500019D02420A0672068016821F001010160E2
:102560002068002505602068456020688560204659
:1025700000F08AF9C4F88050A567E56744F8605F09
:102580000020257570BD012070BD70472DE9F04118
:1025900002680446D0691168936840F60F05284226
:1025A0004FF0000505D186067ED58E067CD5616E7E
:1025B0001BE1994F03F001060F40374374D0C70762
:1025C00009D0CF0507D501271762D4F8802042F043
:1025D0000102C4F8802082070AD5DA0708D02768EC
:1025E00002223A62D4F8802042F00402C4F880202B
:1025F00042070AD5DA0708D0236804221A62D4F801
:10260000802042F00202C4F8802002070CD501F0BD
:102610002002324308D0236808221A62D4F88020AE
:1026200042F00802C4F8802002050BD54A0109D502
:1026300023684FF400621A62D4F8802042F020022E
:10264000C4F88020D4F88020002A35D0800605D533
:10265000880603D5616E09B120468847D4F880000A
:1026600021688968490602D410F0280F26D0204638
:1026700001F09EF82068806840061AD5206808306E
:1026800050E8001F21F0400140E80012002AF5D177
:10269000206F70B161498163206FFEF717FD00283C
:1026A0000AD0206F816B01E00EE02046BDE8F041CA
:1026B00008472046FFF769FFBDE8F0812046FFF795
:1026C00064FFC4F88050F7E7276E2026012F7BD1E6
:1026D000C70679D5CF0677D51020106220688068AC
:1026E000400641D5216F086840680004000CE3D023
:1026F000B4F858208242DFD9A4F85A00086800686C
:1027000080062AD4206850E8001F21F4807140E838
:102710000012002AF6D12068083050E8001F21F08E
:10272000010140E80012002AF5D12068083050E885
:10273000001F21F0400140E80012002AF5D1E667B1
:102740002566216851E8000F20F0100041E80002E2
:10275000002AF6D1206FFEF794FCB4F85800B4F8C4
:102760005A10401A81B22AE0B4F85800B4F85A104E
:10277000401A81B2B4F85A0000289DD000299BD09D
:10278000226852E8000F20F4907042E80003002B0A
:10279000F6D12068083050E8002F22F0010240E80E
:1027A0000023002BF5D1E66725666566226852E8AE
:1027B000000F20F0100042E80003002BF6D1204665
:1027C000FFF739FE78E7FFE7C70209D55B0207D5B7
:1027D0004FF4801010622046BDE8F041FFF76FBE55
:1027E000020606D50A0604D5A16E00297FF45DAF66
:1027F00062E74006E6D54806E4D52046026852E87E
:10280000001F21F0400142E80013002BF6D186673B
:10281000856600F03DFA4FE72001000469360008A4
:1028200010B5040002D0A06F10B107E0012010BD68
:10283000002084F87400204600F05EF82420A06791
:102840002068016821F001010160204600F0E2FFEC
:102850000128ECD0606A10B1204600F073FE2068B9
:10286000416821F4904141602068816821F02A018B
:1028700081602068016841F0010101602046BDE8E7
:10288000104000F0C3BE000010B50446174B0168AD
:1028900017484FF0904299420FD1C16D21F00101CC
:1028A000C1650C211046FEF791FD206FFEF736FC46
:1028B000E06EFEF733FC462012E00E4B994213D136
:1028C000016E21F4804101664FF4C0611046FEF7AD
:1028D0007DFD206FFEF722FCE06EFEF71FFC252039
:1028E000BDE81040FEF760BF10BD00000080004052
:1028F00000100240003801402DE9F04F9DB0044621
:10290000142117A8FDF799FC5C216846FDF795FC9A
:1029100060492068604F002502264FF003084FF001
:10292000904B4FF0100A4FF08009884256D120207A
:1029300000904FF440600B906846FEF7EDFF08B141
:10294000FDF704FFF86D40F00100F865F86D00F048
:1029500001001C90F86C40F00100F864F86C1995C7
:1029600000F001001C900C20CDE917060820CDE9ED
:102970001A8017A95846FEF7CBFD494E47484FF03D
:1029800004083060C6E90185C6E903597561B5617F
:10299000F5614F4630463562FEF76EFC08B1FDF733
:1029A000D5FE2667B4623E4E3C4848361438C6E928
:1029B00003577561B561F561356286E801053046FA
:1029C000FEF75AFC08B1FDF7C1FEE666002211468B
:1029D0004620B462FEF706FF462056E031498842A1
:1029E00055D10120009008956846FEF795FF08B183
:1029F000FDF7ACFE386E40F480403866386E00F467
:102A000080401C90F86C40F00100F864F86C199557
:102A100000F001001C904FF4C060CDE917060720BC
:102A2000CDE91A8017A95846FEF772FD1C4F1E48C3
:102A30009037C8463860C7E90165C7E903597D6129
:102A4000BD61FD6138463D62FEF716FC08B1FDF739
:102A50007DFE2767BC62124F1348D8371438C7E988
:102A600003587D61BD61FD613D6287E841043846E0
:102A7000FEF702FC08B1FDF769FEE76600220121BE
:102A80002520BC62FEF7AEFE2520FEF79EFE1DB09F
:102A900000F00CB8008000400010024080040240AA
:102AA0009C010020003801405800024030BCBDE8C5
:102AB000C08F000030B4C36F202B20D1E1B1DAB158
:102AC00090F87430012B1AD0012380F87430002361
:102AD00003660C4C0368A3420BD05B681B0208D54D
:102AE000046854E8003F43F0806344E80035002D5B
:102AF000F6D130BC00F08EBF012030BC7047022000
:102B0000FBE70000008000400068064A0121904277
:102B100001D1054803E0054A904201D10448017003
:102B20007047000000380140000000200080004095
:102B300004000020704700002DE9F8430446806F30
:102B40001F4616460D4620284FD1CDB1C6B194F888
:102B50007400012849D0012084F874004FF0000867
:102B6000C4F880802120A067FEF7C8FDA4F850605B
:102B70008146A4F85260A068B0F5805F03D004E0FD
:102B80000120BDE8F883206928B12E465FF00005DA
:102B900084F8748010E00026FAE78021204600F0D7
:102BA0008BFFB8B9C6B116F8010B21680885B4F8D7
:102BB0005200401EA4F85200B4F852004B464FF0A9
:102BC000000200970028E8D14FF04001204600F0B5
:102BD00073FF30B10320D4E735F8020BC0F30800CF
:102BE000E3E72020A0670020CBE70220C9E7000030
:102BF00070B50446806F202841D169B362B394F860
:102C0000740001283BD0012084F87400E164A4F82A
:102C10005020A4F852200025C4F880502120A0673D
:102C2000E06ED8B11749C162E16E174813460863D8
:102C3000E16E16484863E06E85632668E16C06F134
:102C40002802E06EFEF778FB40B11020C4F8800047
:102C500004F8745F20206060012070BD216840206E
:102C6000086284F874502068083050E8001F41F072
:102C7000800140E80012002AF5D1002070BD02203A
:102C800070BD000065370008A73700087D360008D2
:102C900070477047FEE708B500200090401C009088
:102CA0007828FBDB08BD000070B5002500F088FB2C
:102CB0000F4E0024012204213046FEF719FDFFF7D4
:102CC000EAFF02213046FEF70EFD40EA4500C5B29C
:102CD000002204213046FEF70BFDFFF7DCFF641CE9
:102CE000E4B2082CE6D300F07FFB284670BD00005C
:102CF0000004004870B5104E05460024280601D592
:102D0000012200E0002202213046FEF7F1FC012200
:102D100004213046FEF7ECFCFFF7BDFF0022042142
:102D20003046FEF7E5FCFFF7B6FF6806641C050EAB
:102D3000E4B2082CE2D370BD0004004810B50D4C7D
:102D4000012202212046FEF7D3FC01220421204665
:102D5000FEF7CEFCFFF79FFF002202212046FEF780
:102D6000C7FCFFF798FF20460022BDE81040042171
:102D7000FEF7BEBC0004004810B50B4C0022022137
:102D80002046FEF7B5FC012204212046FEF7B0FCE8
:102D9000FFF781FF012202212046FEF7A9FCBDE8D2
:102DA0001040FFF778BF00000004004870B5104DD8
:102DB000012202212846FEF79BFC00F001FB0122C4
:102DC00004212846FEF794FCFFF765FF0221284600
:102DD000FEF789FC0446002204212846FEF788FC01
:102DE00000F002FB0CB1002070BD012070BD00009E
:102DF0000004004800EB8100006E00F0F8407047CE
:102E00008068C0F3C00070478068C0F380007047DE
:102E1000C06810F4406F01D0002070470120704757
:102E2000042303EAD15310B518444369C1F3045194
:102E300007248C40A3438A401343436110BD00EB39
:102E40008100016E21F000411143016670470000CE
:102E500010B50B48FFF79AFB09480068C169C943E0
:102E6000C9060BD4102101620548FFF729FBBDE814
:102E70001040042203490248FFF71CBE10BD0000A9
:102E8000940000200A00002030B587B01821684661
:102E9000FDF7D3F9184817490024C0E900148460ED
:102EA0000425C460C0E90445047644760121C1616B
:102EB00080F820408462C46280F83040446380F827
:102EC0003840FDF7F9FE08B1FDF740FC0B480090D3
:102ED0000620CDE901047F200594CDE9030569466C
:102EE0000548FDF735FC002801D0FDF72FFC07B0A1
:102EF00030BD0000000004503000002040002019C8
:102F0000194808B5816C41F001018164816C01F0C0
:102F100001010091816C41F002018164806C00220A
:102F200000F00200009011460E20FEF75BFC0E2020
:102F3000FEF74BFC002211460F20FEF753FC0F203A
:102F4000FEF743FC002211464420FEF74BFC4420D0
:102F5000FEF73BFC002211464520FEF743FCBDE88E
:102F600008404520FEF731BC001002402DE9F04139
:102F700086B014216846FDF760F92748C16C41F01E
:102F80000401C164C16C01F004010591C16C41F000
:102F90000101C164C16C01F001010591C16C41F0F6
:102FA0000201C164C06C4FF0904700F00200059030
:102FB000002201213846FEF79BFBDFF8608043F2D8
:102FC0000646002231464046FEF792FB01250024CA
:102FD0000095CDE90154694638460394FEF798FA06
:102FE0000096CDE90154694640460394FEF790FAF5
:102FF000E802CDE90004694638460294FEF788FAF3
:103000006802CDE90004694640460294FEF780FA62
:1030100006B0BDE8F0810000001002400004004846
:103020000D4810B50B4901604FF416514160002165
:1030300081600C22C160C0E90412816101624162B9
:10304000FFF7EEFB002803D0BDE81040FDF77EBB84
:1030500010BD000000800040940000200D4810B515
:103060000B4901604FF4E1314160002181600C2285
:10307000C160C0E904128161C16101624162FFF770
:10308000CFFB002803D0BDE81040FDF75FBB10BDAB
:103090000038014018010020FEE7FEE770470000FD
:1030A0002DE9F041444C05468846E068002681073A
:1030B00028680DD0E16801F00301814216D1A8B162
:1030C000E0686968C0F30210401C88420ED120E01D
:1030D000012804D0022805D0032807D108E0216880
:1030E000890701E021684905002907DB01265FE027
:1030F0002168890302D421684903F5E7E1686A6819
:103100006FF00F0321F0730103EB0212114301432F
:10311000E160206820F080602060FEF7EFFA07464B
:1031200005E000BFFEF7EAFAC01B022837D8206886
:103130000001F7D4B8F1000F18D0B8F1010F1DD07D
:10314000287D4FF07E41400801EB4060A96840EACD
:1031500001202169194A114008432061206840F08C
:1031600080602060FEF7CAFA07461AE0A868297B4B
:10317000000240EAC1602169114AECE7288A11493E
:10318000400801EB4050A96840EA012021690E4A3D
:10319000E1E700BFFEF7B2FAC01B022801D90326FF
:1031A00006E020680001F5D52069A969084320617F
:1031B0003046BDE8F081000000100240FF80FFF9BA
:1031C000FF80FF070000E0FFFF809FFFF8B51C4D68
:1031D00006460024A86DC00002D5FEF785FB0DE071
:1031E000A86D40F08050A865A86D00F08050009058
:1031F000FEF77AFBA96D21F08051A965B0F5007F3B
:1032000004D0802E07D94FF003040AE0802E08D99D
:10321000A02E01D804E001D1022402E0702E00D1DA
:1032200001240848016821F007012143016000687A
:1032300000F00700A04201D00120F8BD0020F8BD39
:10324000001002400020024010B50348FFF796F836
:1032500002490120087010BDBC02002014000020AB
:1032600070B500242546661E0A48FDF7A7FE3146C4
:103270000848FDF74BFE18B90648FDF719FD044450
:103280000448FDF7DFFE6D1C0A2DEDDB0A20B4FBC0
:10329000F0F070BD3000002010B54FF4007103480D
:1032A000FEF721FA002800D0012010BD00040048DC
:1032B00070B586B0002440F29D654FF46E7601AA89
:1032C00004A9684600F053F8BDF90000A84207D1F0
:1032D000BDF81000302803D1BDF90400B042EED093
:1032E00003AA05A902A800F042F8BDF90800A84207
:1032F00007D1BDF81400302803D1BDF90C00B0424D
:10330000EED0BDF90810BDF900000A1A102A0CDC35
:10331000401A102809DCBDF90C10BDF904000A1A86
:103320000F2A02DC401A0F2800DD012406B02046D7
:1033300070BD41EA002000B20011010502D540F441
:10334000704000B2704770B520252F220024294616
:10335000182000F08FF82A462321182000F08AF860
:103360002246BDE870402121182000F083B87CB5CA
:1033700014460E46054606236A46A821182000F08A
:1033800048F89DF800109DF80100FFF7D2FF288053
:103390009DF802109DF80300FFF7CBFF30809DF8E9
:1033A00004109DF80500FFF7C4FF2080288800F274
:1033B000DC502880208800F6B83020807CBD0000DA
:1033C00000B585B014216846FCF737FF0220009055
:1033D00000200190029069460248FEF799F805B076
:1033E00000BD00000004004800B585B01421684607
:1033F000FCF723FF02200090112001900020029092
:1034000069460248FEF784F805B000BD0004004894
:1034100070472DE9F0411C4615460F460646FFF75A
:103420008DFC7006000EFFF765FCFFF7BFFC00285F
:103430001ED03846FFF75EFCFFF7B8FC002817D017
:10344000FFF77CFC012000EB4600C0B2FFF752FC06
:10345000FFF7ACFC00280BD003E0FFF725FC05F8D4
:10346000010B641EA4B2F8D2BDE8F041FFF784BCA2
:10347000BDE8F08170B515460E460446FFF75EFCC8
:103480006006000EFFF736FCFFF790FC002811D015
:103490003046FFF72FFCFFF789FC00280AD02846AA
:1034A000FFF728FCFFF782FC002803D0BDE870403E
:1034B000FFF762BC70BDFEF727B9000010B596B0EB
:1034C00044216846FCF7B9FE142111A8FCF7B5FEAB
:1034D0004FF40070FEF7B8F908B172B6FEE7FEF7D8
:1034E0000BFA134850F8901F21F0180101601420C6
:1034F0000090012000240290CDE90604802008906D
:103500000A946846FEF77EFC08B172B6FEE70F200B
:10351000CDE9110413941494002111A81594FEF719
:1035200059FB08B172B6FEE7FEF7EEF916B010BD12
:10353000001002400248016841F4700101607047C8
:1035400088ED00E090F82410C90706D001684A68A9
:10355000836A22F400321A434A6090F824108907E3
:1035600006D501684A68C36A22F480321A434A6069
:1035700090F82410490706D501684A68036B22F4C5
:1035800080221A434A6090F82410090706D5016882
:103590004A68436B22F400421A434A6090F82410B0
:1035A000C90606D501688A68836B22F480521A43E3
:1035B0008A6090F82410890606D501688A68C36B72
:1035C00022F400521A438A6090F82410490611D55B
:1035D00001684A68036C22F480121A434A60016C45
:1035E000B1F5801F06D101684A68436C22F4C0021D
:1035F0001A434A6090F82410090606D501684A6803
:10360000806C22F4002202434A607047F8B500261D
:103610000446C0F88060FEF771F80546206800682F
:103620006FF07E47000708D52B4600224FF40011AB
:103630002046009700F040FA60B920680068400713
:103640000AD52B4600224FF480012046009700F057
:1036500033FA08B10320F8BD2020A067E067266692
:1036600084F874600020F8BD10B5806A0021A0F8CD
:103670005A10A0F85210FEF788FF10BD70B5846A8A
:10368000A06FE56F216889684FF00006090606D52E
:10369000212804D1A4F85260204600F0AEF820683A
:1036A0008068400606D5222D04D1A4F85A60204631
:1036B00000F07EF8D4F8800040F01000C4F88000DC
:1036C0002046FEF762FF70BD10B50146806A0968AA
:1036D000096889062DD40021A0F85A10016851E824
:1036E000002F22F4807241E80023002BF6D10168FC
:1036F000083151E8002F22F0010241E80023002B9D
:10370000F5D10168083151E8002F22F0400241E86C
:103710000023002BF5D12021C167016E012908D1BA
:10372000026852E8001F21F0100142E80013002B4C
:10373000F6D1016E012902D0FFF7E6F910BDB0F80D
:103740005810FEF778FE10BD10B5806A016E012991
:1037500002D0FFF7EFF910BDB0F858104908FEF796
:103760006AFE10BD10B50146806A096809688906BD
:1037700016D40021A0F852100168083151E8002F3A
:1037800022F0800241E80023002BF5D1026852E8C4
:10379000001F41F0400142E80013002BF6D110BD9C
:1037A000FFF776FA10BD10B5806AFFF772FA10BD08
:1037B000016851E8002F22F4907241E80023002BA9
:1037C000F6D10168083151E8002F22F0010241E8EA
:1037D0000023002BF5D1016E012908D1026852E8BF
:1037E000001F21F0100142E80013002BF6D1202128
:1037F000C1670021016641667047026852E8001FF8
:1038000021F0C00142E80013002BF6D1202181678E
:10381000704700002DE9F041044601688068226984
:10382000E3691043626900251A431043714F0A6827
:10383000714B1A4002430A6020684168E26821F433
:103840004051114341602168A069B94201D0226A08
:1038500010438A6822F4306202438A606749236811
:1038600067488B420DD1D0F8880010F0030006D0D5
:10387000012847D0022843D0032830D144E0012159
:103880002EE060498B420BD1D0F8880010F00C007C
:1038900034D0042836D0082832D00C281FD133E089
:1038A00059498B420BD1D0F8880010F0300025D058
:1038B000102827D0202823D0302810D124E0BB4264
:1038C0000DD1D0F8880010F4406017D0B0F5806FAB
:1038D00018D0B0F5006F13D0B0F5406F14D01021A0
:1038E0004A4A00264FF40040BB422FD171B1022951
:1038F0000FD004290FD0082973D10FE00021EFE782
:103900000221EDE70421EBE70821E9E7FEF704FADD
:1039100003E0104602E0FEF723FAE8B3626802EB28
:10392000420181425DD8B0EB023F5AD8010E03023A
:103930005008181871410023FCF744FC344AA0F5E4
:10394000407191424DD82168C8604BE0E3694FF661
:10395000EF77834228D1092943D2DFE801F0050837
:103960000B420D4242421000FEF7D6F906E0FEF788
:10397000E5F903E0104602E0FEF7F2F960B141001C
:10398000606801EB5001B1FBF0F0A0F11001B94209
:1039900027D84FF6F07100E024E00140C0F3420068
:1039A00001432068C1601DE009291AD2DFE801F057
:1039B00005080B190D1919191000FEF7ADF906E0ED
:1039C000FEF7BCF903E0104602E0FEF7C9F948B182
:1039D000616800EB5100B0FBF1F0A0F11001B942B9
:1039E00005D9012566662846A666BDE8F08180B245
:1039F000A9E7000000800040F369FFEF00380140B4
:103A00000010024000440040004800400024F40040
:103A1000FFFC0F0070B54165A0F858200025044652
:103A2000C0F880502220E067206FD8B11F49C162E2
:103A3000216F1F4813460863216F1E484863206F9B
:103A40008563666D216832462431206FFDF774FC72
:103A500040B11020C4F8800004F8745F2020A060FA
:103A6000012070BD84F87450206940B1216851E88C
:103A7000000F40F4807041E80002002AF6D120686F
:103A8000083050E8001F41F0010140E80012002A10
:103A9000F5D12068083050E8001F41F0400140E8AF
:103AA0000012002AF5D1002070BD0000C9360008C0
:103AB000493700087D3600082DE9F0479A46174639
:103AC0000E4604464FF000094FF02008089D4AE0DA
:103AD000681C48D0FDF712FEA0EB0A00A8422AD8C5
:103AE0004DB32068016849073DD5C069C043000552
:103AF00039D421684FF400600862206850E8001F44
:103B000021F4D07140E80012002AF6D12068083074
:103B100050E8001F21F0010140E80012002AF5D111
:103B2000C4F87880C4F87C80C4F8808084F87490ED
:103B30000320BDE8F087216851E8000F20F4D07021
:103B400041E80002002AF6D12068083050E8001F42
:103B500021F0010140E80012002AF5D1C4F8788074
:103B6000C4F87C80E2E72068C06936EA000004D02F
:103B70000020B842ACD00020DBE70120F9E70000CC
:103B800010B50B48FEF702FD09480068C169C9433A
:103B9000C9060CD4102101620548FEF791FC0422ED
:103BA00004490348FEF786FF03490120087010BD51
:103BB000180100201500002000000020FEE7000092
:103BC000014A024900F023B8313C00082C000020D3
:103BD0000907090E002804DB00F1E02080F800143A
:103BE000704700F00F0000F1E02080F8141D7047CE
:103BF00002E008C8121F08C1002AFAD170477047B6
:103C0000002001E001C1121F002AFBD170472DE9FD
:103C1000F04116460F460446002503E03946B047FA
:103C2000641C6D1C20780028F8D12846BDE8F0817E
:103C300013B54FF6FF73012269460248FEF77CFF79
:103C400000981CBD180100201CB5FDF765FDFFF7AD
:103C500035FCFFF78BF9FFF753F9FFF7FFF9FFF793
:103C6000DFF9FFF711F9FFF76EFB574D57480026B4
:103C70002E600068016841F01001016004222946AD
:103C80005248FEF717FF524F4FF48064002221463E
:103C90003846FDF72DFD4FF4FA70FDF785FB012244
:103CA00021463846FDF724FD4AA0FFF789FF0B2285
:103CB0004AA14648FEF79CFF40F6B830FDF774FB7A
:103CC00001224FF0904811464046FDF711FDAC1F10
:103CD000FCF7DCFC20780028FAD02670287803282E
:103CE00060D16878012832D16F8802213648FCF70C
:103CF00021FC874228D1002201214046FDF7F8FC33
:103D0000FFF7CAFA6070FFF7ABFAE060E068FCF713
:103D1000D3FBA080F1208DF8000060788DF80100C1
:103D2000F2208DF80200A0888DF803000421684677
:103D3000FCF700FC8DF80400000A8DF8050006224F
:103D400069462248FEF754FF287803282AD168786C
:103D5000022827D16F8802211B48FCF7EBFB874222
:103D600020D1002201214046FDF7C2FCFFF7A0FA56
:103D7000A070F3208DF80000A0788DF801000221DA
:103D80006846FCF7D7FB8DF80200000A8DF80300A7
:103D9000042269460D48FEF72BFF6420FDF704FB63
:103DA000FCF774FC042208490848FEF783FE0A2049
:103DB000FDF7FAFA012211464046FDF799FC0A2068
:103DC000FDF7F2FA84E700000A00002094000020CA
:103DD000000400486C705F5634350A0041542B547F
:103DE00052414E4D443D31000000000000000000F3
:103DF0000102030406070809A0860100400D030024
:103E0000801A060000350C0040420F0080841E001E
:103E100000093D0000127A000024F40000366E0113
:103E20000048E801006CDC0200000000010203040D
:103E3000503E00080000002030000000F03B000869
:103E4000803E000830000020B0060000003C000862
:103E50000000000000000000000000000000000062
:103E60000000000000000000000000000100000051
:103E7000100000000000000000093D0000000000EC
:040000050800018D61
:00000001FF
